******************************************************************************
               TMS320C6x Linker PC v7.2.2                      
******************************************************************************
>> Linked Mon Nov 21 17:06:02 2011

OUTPUT FILE NAME:   <MPAX.out>
ENTRY POINT SYMBOL: "_c_int00"  address: 00809fe0


MEMORY CONFIGURATION

         name            origin    length      used     unused   attr    fill
----------------------  --------  ---------  --------  --------  ----  --------
  VECTORS_MEM           00800000   00000400  00000200  00000200  RWIX
  BOOT_MEM              00800400   00001c00  00000000  00001c00  RWIX
  TEXT_MEM              00802000   0007e000  00011cdc  0006c324  RWIX
  MSMCSRAM0             0c000000   00100000  00000004  000ffffc  RWIX
  MSMCSRAM1             0c100000   00100000  00000000  00100000  RWIX
  MSMCSRAMALIAS_CACHABL 30000000   00100000  00000008  000ffff8  RWIX
  MSMCSRAMALIAS_NONCACH 31000000   00100000  00000004  000ffffc  RWIX
  DATA_ALIAS_L2_MEM     40000000   00100000  00000004  000ffffc  RWIX
  DDR2                  80000000   10000000  00000000  10000000  RWIX


SEGMENT ALLOCATION MAP

run origin  load origin   length   init length attrs members
----------  ----------- ---------- ----------- ----- -------
00800000    00800000    00000200   00000200    r-x
  00800000    00800000    00000200   00000200    r-x .csl_vect
00802000    00802000    000086a0   000086a0    r-x
  00802000    00802000    000086a0   000086a0    r-x .text
0080a6a0    0080a6a0    00008000   00000000    rw-
  0080a6a0    0080a6a0    00004000   00000000    rw- .stack
  0080e6a0    0080e6a0    00004000   00000000    rw- .sysmem
008126a0    008126a0    00000978   00000978    r--
  008126a0    008126a0    00000978   00000978    r-- .const
00813020    00813020    00000700   00000000    rw-
  00813020    00813020    00000700   00000000    rw- .far
00813720    00813720    00000324   00000204    rw-
  00813720    00813720    00000204   00000204    rw- .fardata
  00813924    00813924    00000120   00000000    rw- .cio
00813a44    00813a44    0000009c   0000009c    r--
  00813a44    00813a44    0000009c   0000009c    r-- .switch
00813ae0    00813ae0    000000a8   000000a8    rw-
  00813ae0    00813ae0    00000058   00000058    rw- .bss
  00813b38    00813b38    00000050   00000050    rw- .neardata
00813b88    00813b88    0000015c   0000015c    r--
  00813b88    00813b88    0000015c   0000015c    r-- .cinit
0c000000    0c000000    00000004   00000000    rw-
  0c000000    0c000000    00000004   00000000    rw- .mydata
30000000    30000000    00000008   00000000    rw-
  30000000    30000000    00000008   00000000    rw- .mycachable
31000000    31000000    00000004   00000000    rw-
  31000000    31000000    00000004   00000000    rw- .mynoncachable
40000000    40000000    00000004   00000000    rw-
  40000000    40000000    00000004   00000000    rw- .myaliasL2data


SECTION ALLOCATION MAP

 output                                  attributes/
section   page    origin      length       input sections
--------  ----  ----------  ----------   ----------------
.csl_vect 
*          0    00800000    00000200     
                  00800000    00000200     ti.csl.intc.ae66e : _csl_intcIsrDispatch.oe66e (.csl_vect)

.text      0    00802000    000086a0     
                  00802000    000007a0     xmc_cache_test.obj (.text)
                  008027a0    000005e0     rts6600e_elf.lib : divd.obj (.text:__c6xabi_divd)
                  00802d80    000005c0                      : _printfi.obj (.text:_getarg_diouxp)
                  00803340    000004e0     Interrupt.obj (.text)
                  00803820    000004c0     Exception.obj (.text)
                  00803ce0    000004a0     rts6600e_elf.lib : _printfi.obj (.text:_setfield)
                  00804180    00000480                      : _printfi.obj (.text:_printfi)
                  00804600    000003e0     ti.csl.intc.ae66e : csl_intcHwControl.oe66e (.text:csl_section:intc:CSL_intcHwControl)
                  008049e0    00000300     rts6600e_elf.lib : fputs.obj (.text:fputs)
                  00804ce0    000002e0                      : _printfi.obj (.text:_pproc_fwp)
                  00804fc0    000002c0                      : _printfi.obj (.text:_pproc_fge)
                  00805280    000002a0                      : _printfi.obj (.text:fcvt)
                  00805520    00000280                      : _printfi.obj (.text:ecvt)
                  008057a0    00000280                      : memory.obj (.text:free)
                  00805a20    00000240                      : imath64.obj (.text:__c6xabi_divull)
                  00805c60    00000240                      : _printfi.obj (.text:_pconv_e)
                  00805ea0    00000240     ti.csl.intc.ae66e : csl_intcOpen.oe66e (.text:csl_section:intc:CSL_intcOpen)
                  008060e0    00000220     rts6600e_elf.lib : _printfi.obj (.text:_pproc_diouxp)
                  00806300    00000220                      : _printfi.obj (.text:_pproc_str)
                  00806520    00000200                      : _printfi.obj (.text:_pconv_g)
                  00806720    00000200     ti.csl.intc.ae66e : _csl_intcCombEventDispatcher.oe66e (.text:csl_section:intc:_CSL_intcEvent0Dispatcher)
                  00806920    00000200                       : _csl_intcCombEventDispatcher.oe66e (.text:csl_section:intc:_CSL_intcEvent1Dispatcher)
                  00806b20    00000200                       : _csl_intcCombEventDispatcher.oe66e (.text:csl_section:intc:_CSL_intcEvent2Dispatcher)
                  00806d20    00000200                       : _csl_intcCombEventDispatcher.oe66e (.text:csl_section:intc:_CSL_intcEvent3Dispatcher)
                  00806f20    000001e0                       : _csl_intcDispatcher.oe66e (.text:csl_section:intc:_CSL_intcDispatcher)
                  00807100    000001c0     rts6600e_elf.lib : _printfi.obj (.text:_mcpy)
                  008072c0    000001a0                      : trgdrv.obj (.text:HOSTrename)
                  00807460    000001a0                      : imath40.obj (.text:__c6xabi_divul)
                  00807600    000001a0                      : memory.obj (.text:malloc)
                  008077a0    000001a0                      : setvbuf.obj (.text:setvbuf)
                  00807940    00000180                      : copy_decompress_rle.obj (.text:__TI_decompress_rle_core)
                  00807ac0    00000180                      : autoinit.obj (.text:_auto_init_elf)
                  00807c40    00000180     Exception.obj (.text:retain)
                  00807dc0    00000160     rts6600e_elf.lib : frcmpyd_div.obj (.text:__c6xabi_frcmpyd_div)
                  00807f20    00000160     ti.csl.intc.ae66e : csl_intcInit.oe66e (.text:csl_section:intc:CSL_intcInit)
                  00808080    00000140     ti.csl.ae66e : csl_chip.oe66e (.text:CSL_chipReadReg)
                  008081c0    00000140     rts6600e_elf.lib : _printfi.obj (.text:_pproc_fflags)
                  00808300    00000140     ti.csl.intc.ae66e : _csl_intcIntrEnDisRes.oe66e (.text:csl_section:intc)
                  00808440    00000140     rts6600e_elf.lib : fputc.obj (.text:fputc)
                  00808580    00000140                      : lowlev.obj (.text:getdevice)
                  008086c0    00000120                      : _printfi.obj (.text:_ltostr)
                  008087e0    00000120                      : fclose.obj (.text:fclose)
                  00808900    00000100                      : trgdrv.obj (.text:HOSTlseek)
                  00808a00    00000100                      : _io_perm.obj (.text:_wrt_ok)
                  00808b00    00000100                      : cpy_tbl.obj (.text:copy_in)
                  00808c00    000000e0                      : trgdrv.obj (.text:HOSTopen)
                  00808ce0    000000e0                      : _printfi.obj (.text:_div)
                  00808dc0    000000e0                      : atoi.obj (.text:atoi)
                  00808ea0    000000e0                      : lowlev.obj (.text:close)
                  00808f80    000000e0                      : copy_zero_init.obj (.text:decompress:ZI:__TI_zero_init)
                  00809060    000000e0                      : exit.obj (.text:exit)
                  00809140    000000e0                      : memset.obj (.text:memset)
                  00809220    000000c0                      : trgdrv.obj (.text:HOSTread)
                  008092e0    000000c0                      : trgdrv.obj (.text:HOSTunlink)
                  008093a0    000000c0                      : trgdrv.obj (.text:HOSTwrite)
                  00809460    000000c0                      : divu.obj (.text:__divu)
                  00809520    000000c0                      : fopen.obj (.text:_cleanup)
                  008095e0    000000c0                      : fflush.obj (.text:_doflush)
                  008096a0    000000c0     ti.csl.intc.ae66e : csl_intcPlugEventHandler.oe66e (.text:csl_section:intc:CSL_intcPlugEventHandler)
                  00809760    000000c0     rts6600e_elf.lib : fseek.obj (.text:fseek)
                  00809820    000000c0                      : lowlev.obj (.text:lseek)
                  008098e0    000000c0                      : ltoa.obj (.text:ltoa)
                  008099a0    000000c0                      : lowlev.obj (.text:write)
                  00809a60    000000a0                      : trgdrv.obj (.text:HOSTclose)
                  00809b00    000000a0                      : _printfi.obj (.text:_ecpy)
                  00809ba0    000000a0                      : _printfi.obj (.text:_fcpy)
                  00809c40    000000a0                      : _printfi.obj (.text:_pconv_f)
                  00809ce0    000000a0                      : lowlev.obj (.text:finddevice)
                  00809d80    000000a0                      : memcpy64.obj (.text:memcpy)
                  00809e20    000000a0                      : memory.obj (.text:minsert)
                  00809ec0    000000a0                      : memory.obj (.text:mremove)
                  00809f60    00000080                      : llshift.obj (.text:__c6xabi_llshl)
                  00809fe0    00000080                      : boot.obj (.text:_c_int00)
                  0080a060    00000080                      : memory.obj (.text:_minit)
                  0080a0e0    00000080                      : printf.obj (.text:printf)
                  0080a160    00000080                      : trgmsg.obj (.text:readmsg)
                  0080a1e0    00000080                      : lowlev.obj (.text:unlink)
                  0080a260    00000060                      : llshift.obj (.text:__c6xabi_llshru)
                  0080a2c0    00000060                      : imath64.obj (.text:_subcull)
                  0080a320    00000060                      : memccpy.obj (.text:memccpy)
                  0080a380    00000060                      : trgmsg.obj (.text:writemsg)
                  0080a3e0    00000040     ti.csl.ae66e : csl_cpIntcGetBaseAddress.oe66e (.text:CSL_CPINTC_open)
                  0080a420    00000040     rts6600e_elf.lib : isinf.obj (.text:__c6xabi_isinf)
                  0080a460    00000040                      : _printfi.obj (.text:__c6xabi_isnan)
                  0080a4a0    00000040                      : divd.obj (.text:__c6xabi_isnan)
                  0080a4e0    00000040                      : args_main.obj (.text:_args_main)
                  0080a520    00000040                      : fputs.obj (.text:puts)
                  0080a560    00000020                      : negll.obj (.text:__c6xabi_negll)
                  0080a580    00000020                      : tdeh_init.obj (.text:__tdeh_init)
                  0080a5a0    00000020                      : _lock.obj (.text:_nop)
                  0080a5c0    00000020                      : printf.obj (.text:_outc)
                  0080a5e0    00000020                      : printf.obj (.text:_outs)
                  0080a600    00000020                      : exit.obj (.text:abort)
                  0080a620    00000020     ti.csl.intc.ae66e : csl_intcHookIsr.oe66e (.text:csl_section:intc:CSL_intcHookIsr)
                  0080a640    00000020                       : _csl_intcNmiDummy.oe66e (.text:csl_section:intc)
                  0080a660    00000020     rts6600e_elf.lib : copy_decompress_none.obj (.text:decompress:none:__TI_decompress_none)
                  0080a680    00000020                      : copy_decompress_rle.obj (.text:decompress:rle24:__TI_decompress_rle24)

.stack     0    0080a6a0    00004000     UNINITIALIZED
                  0080a6a0    00000008     rts6600e_elf.lib : boot.obj (.stack)
                  0080a6a8    00003ff8     --HOLE--

.sysmem    0    0080e6a0    00004000     UNINITIALIZED
                  0080e6a0    00000008     rts6600e_elf.lib : memory.obj (.sysmem)
                  0080e6a8    00003ff8     --HOLE--

.const     0    008126a0    00000978     
                  008126a0    000003c4     xmc_cache_test.obj (.const:.string)
                  00812a64    000003a0     Exception.obj (.const:.string)
                  00812e04    00000002     rts6600e_elf.lib : fputs.obj (.const:.string)
                  00812e06    0000000a     --HOLE-- [fill = 0]
                  00812e10    00000101                      : ctype.obj (.const:_ctypes_)
                  00812f11    00000003     --HOLE-- [fill = 0]
                  00812f14    000000d4     Interrupt.obj (.const:.string)
                  00812fe8    00000023     rts6600e_elf.lib : _printfi.obj (.const:.string)
                  0081300b    00000005     --HOLE-- [fill = 0]
                  00813010    00000008                      : divd.obj (.const:initial_approx$1)

.far       0    00813020    00000700     UNINITIALIZED
                  00813020    00000580     Interrupt.obj (.far)
                  008135a0    000000d8     rts6600e_elf.lib : trgdrv.obj (.far)
                  00813678    00000008     --HOLE--
                  00813680    000000a0                      : defs.obj (.far)

.fardata   0    00813720    00000204     
                  00813720    000000f0     rts6600e_elf.lib : defs.obj (.fardata:_ftable)
                  00813810    00000078                      : lowlev.obj (.fardata:_device)
                  00813888    00000008                      : _lock.obj (.fardata)
                  00813890    00000050                      : lowlev.obj (.fardata:_stream)
                  008138e0    00000010     Interrupt.obj (.fardata:intInfo)
                  008138f0    0000000c     Interrupt.obj (.fardata:cpintcInfo)
                  008138fc    00000004     rts6600e_elf.lib : defs.obj (.fardata)
                  00813900    0000000c     Interrupt.obj (.fardata:handle)
                  0081390c    0000000c     rts6600e_elf.lib : exit.obj (.fardata)
                  00813918    0000000c                      : memory.obj (.fardata)

.cio       0    00813924    00000120     UNINITIALIZED
                  00813924    00000120     rts6600e_elf.lib : trgmsg.obj (.cio)

.switch    0    00813a44    0000009c     
                  00813a44    00000070     ti.csl.ae66e : csl_chip.oe66e (.switch:CSL_chipReadReg)
                  00813ab4    0000001c     ti.csl.intc.ae66e : csl_intcHwControl.oe66e (.switch:CSL_intcHwControl)
                  00813ad0    00000010                       : csl_intcOpen.oe66e (.switch:CSL_intcOpen)

.bss       0    00813ae0    00000058     
                  00813ae0    0000004c     ti.csl.intc.ae66e : _csl_intcResource.oe66e (.bss:csl_section:intc:uninit) [fill = 0]
                  00813b2c    00000008                       : _csl_intcResource.oe66e (.bss:csl_section:intc:init)
                  00813b34    00000004     Interrupt.obj (.bss) [fill = 0]

.neardata 
*          0    00813b38    00000050     
                  00813b38    00000050     Exception.obj (.neardata)

.cinit     0    00813b88    0000015c     
                  00813b88    00000081     (.cinit..fardata.load) [load image, compression = rle]
                  00813c09    00000003     --HOLE-- [fill = 0]
                  00813c0c    00000056     (.cinit..neardata.load) [load image, compression = rle]
                  00813c62    00000002     --HOLE-- [fill = 0]
                  00813c64    0000000c     (__TI_handler_table)
                  00813c70    00000009     (.cinit..bss.load) [load image, compression = rle]
                  00813c79    00000003     --HOLE-- [fill = 0]
                  00813c7c    00000008     (.cinit..far.load) [load image, compression = zero_init]
                  00813c84    00000008     (.cinit..myaliasL2data.load) [load image, compression = zero_init]
                  00813c8c    00000008     (.cinit..mycachable.load) [load image, compression = zero_init]
                  00813c94    00000008     (.cinit..mydata.load) [load image, compression = zero_init]
                  00813c9c    00000008     (.cinit..mynoncachable.load) [load image, compression = zero_init]
                  00813ca4    00000040     (__TI_cinit_table)

.mydata    0    0c000000    00000004     UNINITIALIZED
                  0c000000    00000004     xmc_cache_test.obj (.mydata)

.mycachable 
*          0    30000000    00000008     UNINITIALIZED
                  30000000    00000008     xmc_cache_test.obj (.mycachable)

.mynoncachable 
*          0    31000000    00000004     UNINITIALIZED
                  31000000    00000004     xmc_cache_test.obj (.mynoncachable)

.myaliasL2data 
*          0    40000000    00000004     UNINITIALIZED
                  40000000    00000004     xmc_cache_test.obj (.myaliasL2data)


LINKER GENERATED COPY TABLES

__TI_cinit_table @ 00813ca4 records: 8, size/record: 8, table size: 64
	.fardata: load addr=00813b88, load size=00000081 bytes, run addr=00813720, run size=00000204 bytes, compression=rle
	.neardata: load addr=00813c0c, load size=00000056 bytes, run addr=00813b38, run size=00000050 bytes, compression=rle
	.bss: load addr=00813c70, load size=00000009 bytes, run addr=00813ae0, run size=00000058 bytes, compression=rle
	.far: load addr=00813c7c, load size=00000008 bytes, run addr=00813020, run size=00000700 bytes, compression=zero_init
	.myaliasL2data: load addr=00813c84, load size=00000008 bytes, run addr=40000000, run size=00000004 bytes, compression=zero_init
	.mycachable: load addr=00813c8c, load size=00000008 bytes, run addr=30000000, run size=00000008 bytes, compression=zero_init
	.mydata: load addr=00813c94, load size=00000008 bytes, run addr=0c000000, run size=00000004 bytes, compression=zero_init
	.mynoncachable: load addr=00813c9c, load size=00000008 bytes, run addr=31000000, run size=00000004 bytes, compression=zero_init


LINKER GENERATED HANDLER TABLE

__TI_handler_table @ 00813c64 records: 3, size/record: 4, table size: 12
	index: 0, handler: __TI_decompress_rle24
	index: 1, handler: __TI_decompress_none
	index: 2, handler: __TI_zero_init


GLOBAL SYMBOLS: SORTED ALPHABETICALLY BY Name 

address    name
--------   ----
0080a600   C$$EXIT
0080a3d8   C$$IO$$
00813b3c   CGEM_regs
008033f0   CSL_CPINTC_generateSysInterrupt
0080a3e0   CSL_CPINTC_open
00808080   CSL_chipReadReg
008083b8   CSL_intcGlobalDisable
00808398   CSL_intcGlobalEnable
0080842c   CSL_intcGlobalExcepClear
00808404   CSL_intcGlobalExcepEnable
00808418   CSL_intcGlobalExtExcepEnable
008083f0   CSL_intcGlobalNmiEnable
008083d8   CSL_intcGlobalRestore
0080a620   CSL_intcHookIsr
00804600   CSL_intcHwControl
00807f20   CSL_intcInit
00808350   CSL_intcInterruptClear
00808330   CSL_intcInterruptDisable
00808310   CSL_intcInterruptEnable
0080836c   CSL_intcInterruptRestore
00808360   CSL_intcInterruptSet
00805ea0   CSL_intcOpen
008096a0   CSL_intcPlugEventHandler
00808384   CSL_intcQueryInterruptStatus
00803a40   EXC_external
00803bc0   EXC_internal
00803ca8   EXC_nmi
00803cc4   EXC_swgen
008134c0   EventRecord
00803820   Exception_cfg
00807c40   Exeception_ISR
00809a60   HOSTclose
00808900   HOSTlseek
00808c00   HOSTopen
00809220   HOSTread
008072c0   HOSTrename
008092e0   HOSTunlink
008093a0   HOSTwrite
00802780   MEMORY_PROTECT_ISR
008130c0   Record
00813b38   XMC_regs
00813b2c   _CSL_intcAllocMask
00813ae0   _CSL_intcCpuIntrTable
00806f20   _CSL_intcDispatcher
00806720   _CSL_intcEvent0Dispatcher
00806920   _CSL_intcEvent1Dispatcher
00806b20   _CSL_intcEvent2Dispatcher
00806d20   _CSL_intcEvent3Dispatcher
00813b28   _CSL_intcEventHandlerRecord
00813b30   _CSL_intcEventOffsetMap
00808300   _CSL_intcIvpSet
0080a640   _CSL_intcNmiDummy
00813b24   _CSL_intcNumEvents
00800000   _CSL_intcVectorTable
00813924   __CIOBUF_
00813ca4   __TI_CINIT_Base
00813ce4   __TI_CINIT_Limit
00813c64   __TI_Handler_Table_Base
00813c70   __TI_Handler_Table_Limit
0080e6a0   __TI_STACK_END
00004000   __TI_STACK_SIZE
00813ae0   __TI_STATIC_BASE
00004000   __TI_SYSMEM_SIZE
00000001   __TI_args_main
0080a660   __TI_decompress_none
0080a680   __TI_decompress_rle24
00813914   __TI_enable_exit_profile_output
ffffffff   __TI_pprof_out_hndl
ffffffff   __TI_prof_data_size
ffffffff   __TI_prof_data_start
00808f80   __TI_zero_init
ffffffff   __binit__
008027a0   __c6xabi_divd
00809460   __c6xabi_divu
00807460   __c6xabi_divul
00805a20   __c6xabi_divull
00807dc0   __c6xabi_frcmpyd_div
0080a420   __c6xabi_isinf
00809f60   __c6xabi_llshl
0080a260   __c6xabi_llshru
0080a560   __c6xabi_negll
ffffffff   __c_args__
00809460   __divu
0080a580   __tdeh_init
0080a4e0   _args_main
00807ac0   _auto_init_elf
00809fe0   _c_int00
00809520   _cleanup
0081390c   _cleanup_ptr
00812e10   _ctypes_
008095e0   _doflush
00813910   _dtors_ptr
008138fc   _ft_end
00813720   _ftable
00813888   _lock
0080a060   _minit
0080a5a0   _nop
00804180   _printfi
0080a6a0   _stack
0080a2c0   _subcull
0080e6a0   _sys_memory
00813680   _tmpnams
0081388c   _unlock
00808a00   _wrt_ok
0080a600   abort
00808dc0   atoi
ffffffff   binit
00813b40   boot_cfg_regs
00808ea0   close
00813020   context
00808b00   copy_in
00813590   coreVector
00813b44   cpIntc0Regs
00813b48   cpIntc1Regs
008138f0   cpintcInfo
00809060   exit
008087e0   fclose
00808440   fputc
008049e0   fputs
008057a0   free
00809760   fseek
00813b58   gEDMACC0Regs
00813b5c   gEDMACC1Regs
00813b60   gEDMACC2Regs
00813900   handle
00813550   hintc
0080346c   initCPINTC
008138e0   intInfo
0080340c   intcInit
008134d0   intcObj
00809820   lseek
008098e0   ltoa
00802380   main
00807600   malloc
0080a320   memccpy
00809d80   memcpy
00803950   memory_protection_exception
00809140   memset
40000000   myL2Var_Alias
0c000000   myVariable
30000004   myVariableMSMC_cacheable
31000000   myVariableMSMC_noncacheable
30000000   myVariable_Alias
00813b4c   pllc_regs
0080a0e0   printf
00813b50   pscRegs
00808440   putc
0080a520   puts
0080a160   readmsg
008035c8   registerInterrupt
0080a1e0   remove
008077a0   setvbuf
00813b54   srioRegs
00813b34   state
00813b64   timer0Regs
00813b68   timer1Regs
00813b6c   timer2Regs
00813b70   timer3Regs
00813b74   timer4Regs
00813b78   timer5Regs
00813b7c   timer6Regs
00813b80   timer7Regs
00813b84   timer8Regs
0080a1e0   unlink
008099a0   write
0080a380   writemsg


GLOBAL SYMBOLS: SORTED BY Symbol Address 

address    name
--------   ----
00000001   __TI_args_main
00004000   __TI_STACK_SIZE
00004000   __TI_SYSMEM_SIZE
00800000   _CSL_intcVectorTable
00802380   main
00802780   MEMORY_PROTECT_ISR
008027a0   __c6xabi_divd
008033f0   CSL_CPINTC_generateSysInterrupt
0080340c   intcInit
0080346c   initCPINTC
008035c8   registerInterrupt
00803820   Exception_cfg
00803950   memory_protection_exception
00803a40   EXC_external
00803bc0   EXC_internal
00803ca8   EXC_nmi
00803cc4   EXC_swgen
00804180   _printfi
00804600   CSL_intcHwControl
008049e0   fputs
008057a0   free
00805a20   __c6xabi_divull
00805ea0   CSL_intcOpen
00806720   _CSL_intcEvent0Dispatcher
00806920   _CSL_intcEvent1Dispatcher
00806b20   _CSL_intcEvent2Dispatcher
00806d20   _CSL_intcEvent3Dispatcher
00806f20   _CSL_intcDispatcher
008072c0   HOSTrename
00807460   __c6xabi_divul
00807600   malloc
008077a0   setvbuf
00807ac0   _auto_init_elf
00807c40   Exeception_ISR
00807dc0   __c6xabi_frcmpyd_div
00807f20   CSL_intcInit
00808080   CSL_chipReadReg
00808300   _CSL_intcIvpSet
00808310   CSL_intcInterruptEnable
00808330   CSL_intcInterruptDisable
00808350   CSL_intcInterruptClear
00808360   CSL_intcInterruptSet
0080836c   CSL_intcInterruptRestore
00808384   CSL_intcQueryInterruptStatus
00808398   CSL_intcGlobalEnable
008083b8   CSL_intcGlobalDisable
008083d8   CSL_intcGlobalRestore
008083f0   CSL_intcGlobalNmiEnable
00808404   CSL_intcGlobalExcepEnable
00808418   CSL_intcGlobalExtExcepEnable
0080842c   CSL_intcGlobalExcepClear
00808440   fputc
00808440   putc
008087e0   fclose
00808900   HOSTlseek
00808a00   _wrt_ok
00808b00   copy_in
00808c00   HOSTopen
00808dc0   atoi
00808ea0   close
00808f80   __TI_zero_init
00809060   exit
00809140   memset
00809220   HOSTread
008092e0   HOSTunlink
008093a0   HOSTwrite
00809460   __c6xabi_divu
00809460   __divu
00809520   _cleanup
008095e0   _doflush
008096a0   CSL_intcPlugEventHandler
00809760   fseek
00809820   lseek
008098e0   ltoa
008099a0   write
00809a60   HOSTclose
00809d80   memcpy
00809f60   __c6xabi_llshl
00809fe0   _c_int00
0080a060   _minit
0080a0e0   printf
0080a160   readmsg
0080a1e0   remove
0080a1e0   unlink
0080a260   __c6xabi_llshru
0080a2c0   _subcull
0080a320   memccpy
0080a380   writemsg
0080a3d8   C$$IO$$
0080a3e0   CSL_CPINTC_open
0080a420   __c6xabi_isinf
0080a4e0   _args_main
0080a520   puts
0080a560   __c6xabi_negll
0080a580   __tdeh_init
0080a5a0   _nop
0080a600   C$$EXIT
0080a600   abort
0080a620   CSL_intcHookIsr
0080a640   _CSL_intcNmiDummy
0080a660   __TI_decompress_none
0080a680   __TI_decompress_rle24
0080a6a0   _stack
0080e6a0   __TI_STACK_END
0080e6a0   _sys_memory
00812e10   _ctypes_
00813020   context
008130c0   Record
008134c0   EventRecord
008134d0   intcObj
00813550   hintc
00813590   coreVector
00813680   _tmpnams
00813720   _ftable
00813888   _lock
0081388c   _unlock
008138e0   intInfo
008138f0   cpintcInfo
008138fc   _ft_end
00813900   handle
0081390c   _cleanup_ptr
00813910   _dtors_ptr
00813914   __TI_enable_exit_profile_output
00813924   __CIOBUF_
00813ae0   _CSL_intcCpuIntrTable
00813ae0   __TI_STATIC_BASE
00813b24   _CSL_intcNumEvents
00813b28   _CSL_intcEventHandlerRecord
00813b2c   _CSL_intcAllocMask
00813b30   _CSL_intcEventOffsetMap
00813b34   state
00813b38   XMC_regs
00813b3c   CGEM_regs
00813b40   boot_cfg_regs
00813b44   cpIntc0Regs
00813b48   cpIntc1Regs
00813b4c   pllc_regs
00813b50   pscRegs
00813b54   srioRegs
00813b58   gEDMACC0Regs
00813b5c   gEDMACC1Regs
00813b60   gEDMACC2Regs
00813b64   timer0Regs
00813b68   timer1Regs
00813b6c   timer2Regs
00813b70   timer3Regs
00813b74   timer4Regs
00813b78   timer5Regs
00813b7c   timer6Regs
00813b80   timer7Regs
00813b84   timer8Regs
00813c64   __TI_Handler_Table_Base
00813c70   __TI_Handler_Table_Limit
00813ca4   __TI_CINIT_Base
00813ce4   __TI_CINIT_Limit
0c000000   myVariable
30000000   myVariable_Alias
30000004   myVariableMSMC_cacheable
31000000   myVariableMSMC_noncacheable
40000000   myL2Var_Alias
ffffffff   __TI_pprof_out_hndl
ffffffff   __TI_prof_data_size
ffffffff   __TI_prof_data_start
ffffffff   __binit__
ffffffff   __c_args__
ffffffff   binit

[166 symbols]
